:020000040000FA
:060000000219FD020310CD
:03001300020501E2
:03001B0002008D53
:03002B000202D5F9
:03005B000205108B
:030073000202FD89
:100080000406080C10182030406080A0C0C2AFC227
:10009000A853E6EFC28E856B8BC0D0D2D3C0E0C030
:1000A000F0C2CAA8CCA9CDD2CAD2AF758A00C3E823
:1000B000956CF8E9956DF9C3E913F9E813F8E5666D
:1000C0006007C3E913F9E813F8E97025E8956E4075
:1000D00020956E501CE582B410177C007B007A00DE
:1000E0007908900000A86AE5667004C3E813F80177
:1000F000FA900000D2A8D2AA61BAE0FDC39CC398CE
:1001000040EF98EB33FB0582E0FCC39DC39840E1D0
:1001100098EB33FB0582E0FDC39CC39840D398EB7A
:1001200033FB0582E0FCC39DC39840C598EB33FBCD
:100130000582E0FDC39CC39840B798EB33FB058272
:10014000E0FCC39DC39840A998EB33FB0582E0FD1A
:10015000C39CC398409B98EB33FB0582E0FCC39D96
:10016000C398408D98EB33FB05822175900000D237
:10017000A8D2AA61BAE0FDC39CC39840EF98EA33C5
:10018000FA0582E0FCC39DC39840E198EA33FA0582
:1001900082E0FDC39CC39840D398EA33FA0582E01D
:1001A000FCC39DC39840C598EA33FA0582E0FDC3BD
:1001B0009CC39840B798EA33FA0582E0FCC39DC31C
:1001C0009840A998EA33FA0582E0FDC39CC39840A1
:1001D0009B98EA33FA0582E0FCC39DC398408D9852
:1001E000EA33FA0582EBC46B6A54F0F9EAC454F0BE
:1001F000C3996009900000D2A8D2AA61BAEBF4C4F6
:1002000054F0F9EAF4C4540F49FAEBF4C4540FFB68
:10021000C3EAF99460FAEB9400FB5020C3E97B0039
:100220007A0079006016C3135006F9C39552600A2C
:10023000E9F552755300790080020553303A27C31F
:10024000EA94D0F8EB9407F9400BE8FAE9FB203583
:1002500009D235415A303502C235203902B235C390
:10026000EA33FAEB33FBEB2B3B3BF9C3EB13FBEA33
:1002700013FAEA29FAEB3400FB30E3047AFF7BFF40
:10028000E5255403601B202A18E55D33F9EB700760
:10029000C3E99A4002E9FAE53CC4332AFAEB340098
:1002A000FBC3EA33C4540FF8EB33C454F048F8707E
:1002B00005EA60027801C3EB13FBEA13FA90000031
:1002C000D2A8D2AAE52260021522819E900000D217
:1002D000A8D2AA61BAC0D0C0E0C2CF0541E5236070
:1002E000021523C3E554600575550041F8E5552412
:1002F00001F55550037555FFD0E0D0D032C2AF5351
:10030000E67F7592FA7593FFC22053917FD2AF3288
:10031000C0E0E58A303408856B8BF0A3D0E032D0A2
:10032000E0C2AF53E6EFC0D0C0E0C0F0D2D3D2AF4E
:100330005388EFA88AA98C758A00758C00438810B1
:1003400030331FE8C4540FFAE9C454F04AFAC31317
:100350002AFAC3E833F8E933F9E82AFAE93403FB67
:1003600061AB30320FC3E833E933FAE82AFAE934F3
:1003700000FB61AB303115E875F056A4AAF0E975C1
:10038000F056A42AFAC5F03400FB61ABE875F02BF7
:10039000A4AAF0E975F02BA42AFAC5F03400C3131F
:1003A000FBEA13FAC3EB13FBEA13FAC3EB9409500D
:1003B00009C3EA949AEB940350160522E5227002D1
:1003C0001522C3E5229432500281F475540081F75E
:1003D000E522600215223036067C007D0461EAAC1D
:1003E00031AD32303A04AC33AD34C3EA9CFAEB9D04
:1003F000FB9208AE60AF61303A425007203509D217
:10040000358108303502C235303504AE62AF632025
:100410003902B235C3EA33FAEB33FBA208500AEAD9
:10042000F42401FAEBF43400FBC3EA9428FAEB94C9
:1004300000FB501478007A007B008148A208500825
:1004400078007A007B00819EE52554036019202AFC
:1004500016E55DF9EB7007C3E99A4002E9FAE53C5D
:10046000C42AFAEB3400FBEA8EF0A4F9AAF0EB8E72
:10047000F0A42AFAC5F03400FBC3EB13FDEA13F82D
:100480000FEF146004C3E833F8C3E933EA33FAEB3F
:1004900033FBDFEDEB30E20678FF7AFF7B03885415
:1004A000D230E86003755500C3E55BFC955C400203
:1004B000AC5CC3EC95545008EC75F004A4FAABF0B6
:1004C000EAF4F8EBF45403F98856895775230AE5E2
:1004D0005A30E110D0F0D0E0D0D053F7DF43F740EE
:1004E00043E61032D0F0D0E0D0D053D8FE43DA014A
:1004F00043E6103275230AD0F0D0E0D0D043E610A6
:1005000032C2AAD28EC2CA85CC6C85CD6DD2CA3217
:10051000C2AFC0D0C0E0D2D38556FB8557FC85570B
:100520005A53F7BF53DAFED2A8303402D2AA53E6A8
:10053000EF53F7DF53D8FED0E0D0D0D2AF327901FD
:10054000801479038010790A800C791E8008796400
:10055000800479C880007817E4D5E0FDD8FAD9F690
:100560002278FF20282879A1E76023E548601F74DE
:10057000FF8548F084853FF030290375F005A4F825
:10058000C5F0600278FFC3E8955D5002A85D885C05
:1005900022C3E54794E4E5489400E55C500314A1C8
:1005A000A2046002F55C2275E89022055EC3E55E58
:1005B0009408405330EDF4A8BDA9BE755E00E9FA79
:1005C00079A0E76041EA7006E55F6018800CC3E837
:1005D000955F600EE55F5005600A1480070460FABD
:1005E0008002E55FF55FC39569401B755BC0C394EE
:1005F000044013755B80C39404400B755B40C39447
:10060000044003755B0022E55B2410500274FFF583
:100610005B22743279A687F0A4C5F0A2F733F55DAA
:10062000227547007548F022C2AFC2CAA8CCA9CD36
:10063000AA4130CF010AD2CAD2AFAB42AC43884202
:100640008943C3E89BF8E99C202808F9302C02E193
:1006500038C191AD448A44F9EA9DFA600678FF7981
:10066000FFC176AE45AF468B458C46A842A943C331
:10067000E89EF8E99FF9C3E54813FBE54713FAE85C
:100680002AF547E93BF54850067547FF7548FFC115
:10069000DEAA47AB48AC47AD487E047F02C3EB946B
:1006A00004400D1E1FC3EB940840052029021E1FA5
:1006B000C3ED13FDEC13FCDEF7C3EA9CFAEB9DFBE4
:1006C000EF6009C3E913F9E813F8DFF7EA28FAEB5A
:1006D00039FB8A478B4850067BFF8B478B48C3EB1F
:1006E00094025002D22C3028047F03E1097892E66C
:1006F000FFC3E53D948240110FC3E53D94A0400146
:100700000FC3EF940640027F057E02E548C4540FF4
:10071000F9E548C454F0F8E547C4540F28F8C3E895
:100720009EFAE99400FB4009C3EA9401EB9400505F
:10073000047A01E4FB020784AA47AB48EBC4FEEA53
:10074000C4540F4EFCC3EA9CFAEB9400FBC3E813BD
:10075000C313F8EA28FAEB3400FB8A478B48C3EB53
:1007600094024002C22C7802EBC4FE7B00EAC4541F
:100770000F4EFAC3EA98FA4005C3940150027A0179
:100780007892E6FF302002E184854E92854F93D225
:100790002043E680C3E49AF8E49BF9302C03020876
:1007A00012E8FAE9FBD3E913FDE813FC884E894F00
:1007B000C3EF94036038EF20E00CE82CF8E93DF932
:1007C000ECFAEDFB8013E828F8E939F9C3E82401D5
:1007D000F8E93400F97AFF7BFFC3EF9403400F8AF6
:1007E000508B51884A894B8C4C8D4D02084788505C
:1007F00089518A4A8B4B8C4C8D4D3028127550F0A4
:100800007551FF754CF0754DFF754EF0754FFF0239
:100810000847E8FAD3E813FC884EC3EF940360213D
:10082000EF20E007E82CF8ECFA0132E8282401F880
:100830007AFFC3EF940340098A50884A8C4C02081F
:100840004788508A4A8C4C3020020147753A02D2C0
:100850002043E680E52554036034A847A948C3E94E
:1008600013F9E813F8C3E913F9E813F8302804E999
:100870002440F9C2AF53E67F759100C3E498F59424
:10088000E499F595759104D22043E680D2AF22D247
:1008900021754900752000302B0375204001ADD231
:1008A00021754900752040302B03752000780179AF
:1008B00001202C20E52554036002C2217914E5486B
:1008C000C313700104F8C394144002781430280450
:1008D000781B791B202010E549600C302803D53A9D
:1008E00004D2222154114F0549E59B5440B5200202
:1008F000213E30280908C3E89940011801D420217D
:100900000A08C3E899400201AD01D4C22153E67F31
:10091000759100302C117594007595F8759104D27D
:100920002043E6800208ADE5487EFFC3334005C39F
:10093000334001FEC3E49E759400F595211CC3E588
:10094000399401500201AD30210201ADD80221528B
:1009500001D4C222C2AF53E67F75910085509485C1
:100960005195759104854A92854B93D22043E68038
:10097000D2AFE525540360072029020539801030E5
:10098000220D202B0A20210715811581021399229F
:1009900078003021027801E53D75F007A4F9E5F013
:1009A00028F5F0E9A2F013A2F113A2F213F53DC36A
:1009B00094785003753D78C3E53D953E4009C2915A
:1009C000C293C29575D57F30200221C7854C928590
:1009D0004D93D22043E68022203814C2AFC293C286
:1009E00090D291D29575D56FD2AF759F2041D8C264
:1009F000AFC293C294D295D29175D57ED2AF759F76
:100A00002041D8203814C2AFC295D29375D57BC28D
:100A100090D291D2AF759F3041D8C2AFC291D293DC
:100A200075D57BC294D295D2AF759F1041D820382E
:100A300014C2AFC291C294D295D29375D57BD2AF76
:100A4000759F1041D8C2AFC295C290D291D2937512
:100A5000D57BD2AF759F3041D8203814C2AFC29336
:100A6000D29175D57EC294D295D2AF759F20806801
:100A7000C2AFC293D29575D56FC290D291D2AF75E5
:100A80009F208054203814C2AFC295C292D293D214
:100A90009175D57ED2AF759F30803DC2AFC291C2F5
:100AA00092D293D29575D56FD2AF759F10802920C1
:100AB0003814C2AFC291D29575D56FC292D293D27B
:100AC000AF759F108012C2AFC295D29175D57EC20C
:100AD00092D293D2AF759F30227A147B7880127AAB
:100AE000107B8C800C7A0D7BB480067A0B7BC880DF
:100AF00000E564D5E001227902E4C293D5E0FDD29D
:100B000092D293D5E0FDC293D5E0FDC292D293D5A7
:100B1000E0FDE920E004D290D29130E004D294D2FA
:100B200095E564D5E0FDE920E002C29130E002C223
:100B3000957496D5E0FDD9C1EAF8D5E0FDD8FBDB88
:100B4000B0C29322C291C293C295C291C293C29580
:100B500075D57F22788076FF0876FF0876FF0876C5
:100B6000FF0876FF0876FF0876090876FF08760109
:100B7000788C76010876FF0876FF0876FF0876FF06
:100B80000876FF0876030876FF0876FF0876FF08E8
:100B900076250876D00876280876500876040876F8
:100BA000FF0876020876FF08767A0876FF0876074F
:100BB0000876010876FF0876FF087600087600229E
:100BC000FA75F00CA4ABF0EAC333F8740133F9E81A
:100BD000C333F8E933F9E8C32BF8E93400F9227894
:100BE00088E6C39403D23A5002C23AC238E630E1F2
:100BF00002D238A23892397886E614900080937831
:100C0000A6F67886E6F53FC394025003753F027856
:100C10009CE6753EFFB40203753EA0B40303753E27
:100C20008278A0E6F8600674282409D8FCF5697873
:100C300096E671C088318932789EE671C088338922
:100C4000347897E671C08835893671442230361180
:100C50007A007B007CFF7D007E0091B38B618A600F
:100C600022303A227896E6FA7B00789EE6FC7D00F8
:100C7000C3EA33FAEB33FBC3EC33FCED33FD7E0AFE
:100C800091B38B638A627896303A02789EE6FA7B5B
:100C9000007897E6FC7D007E00303A10C3EA33FA14
:100CA000EB33FBC3EC33FCED33FD7E0A91B38B6178
:100CB0008A6022C3EC9EFCED9400FDC3EC9AFCED2F
:100CC0009BFDC3EC9423ED940050047C237D00C372
:100CD000EC94FFED940140047CFF7D017BFF0B7AD7
:100CE000000AEA7009C3EC33FCED33FD81DEEC8AC7
:100CF000F0A4AEF0ED8AF0A42E947C40E4EAF46017
:100D0000DD22D236914D12054A12054A7A007B0047
:100D10007C10120542E5542AFA74003BFBDCF37C9C
:100D200004C3EB13FBEA13FADCF7FFEB60027FFF6F
:100D3000C236914D2278A5E6F95403D2867002C2DC
:100D400086E9540CD2877002C287E95430D296707B
:100D500002C296E954C0700022756700756800757C
:100D600097DE7597AD7581C043FF8075EF0675A955
:100D700000714475803F75F1F075A4C075803F75B2
:100D8000D4FF75900075F27F75A57F75900075D5BD
:100D90007F75A60175E34075E202C291C293C295C8
:100DA00012054EC290D291C292D293C294D29512A1
:100DB000053EC291C293C2957144E4F8F6D8FD7124
:100DC000541213D478988664753001C2AF1205525C
:100DD00051D912054A51DF12054A51E512054AB1AF
:100DE00035C2AF75670075680078FA79FA30850703
:100DF000D9FBD8F7021C0071DF914D789886647199
:100E00004475E405758811758E0475890975C804E3
:100E100075910475D84075D90875F782759E00756F
:100E2000960275DA4A75DB0075A82175E69075B8EB
:100E300001759B80759D0075D10C75BC5975BB10F3
:100E400075E88075B20112053ED2AF753C00C23024
:100E5000120552C231C232C233C2347552007553C8
:100E60000075220012054EC3E522940A5002E138B3
:100E7000D23175220012054EC3E522940A5002E1D8
:100E800038C231D23275220012054EC3E522940ACF
:100E90005002E13875E4D5758851758E017589AABF
:100EA000758C00758D00C2A9D2ABD2AA756BC075C6
:100EB0006A14756E50C232D23475220A12054E750C
:100EC0006A10C3E522940A75520075530040697593
:100ED0008E0C756B80756A28756E2875220A12054E
:100EE0004E756A20C3E522940A755200755300407E
:100EF00047758E0C756BC0756A14756E1475220A71
:100F000012054E756A10C3E522940A755200755396
:100F100000402575E405758811758E04758909D220
:100F2000A9C2ABC2AAC234D23375220012054EC385
:100F3000E522940A4002A1E1120542203003020D8D
:100F4000E1C2AF51D951D951D9D2AF120552203493
:100F500003303A03020FF8120542788CE6C394017D
:100F60005003020FF8E530C394015003020FF875E7
:100F700067A57568F17F02D236914D12054EC2AF5A
:100F8000C236914DC3E554947FD2AF406B12053EFB
:100F9000C2AF51EBD2AFDFDFB102C3EF7897F612E9
:100FA00005521214C17F0AD236914D12054EC2AFBE
:100FB000C236914DC3E554947FD2AF50E812053E3E
:100FC000C2AF51D912054651D9D2AFDFDAB102EF23
:100FD00024037896F6F87997E7C394234003985052
:100FE00006E824237897F612055212141B1214F007
:100FF00012054E914D020DE17567007568001205EE
:101000004EC3E55494014003020F4EC2AF120AEBE7
:10101000120AEB120AEBD2AF120552753000E4F55A
:1010200037F5380537E537F4703F0538789AE678B4
:1010300019146012783214600D787D14600878FA03
:10104000146003753800C3E53898401D120B441234
:10105000053E153875370078998664C2AF120AEBE1
:10106000D2AF7898866412054E120546E5237003C8
:10107000020DE1C3E5549401500AC3E552940150B6
:101080001602102312054EE5237003020DE175527E
:1010900000755300021239C3E55294017017C2AFB4
:1010A000120B4478998664120AD978988664D2AF74
:1010B00012054E412BC3E55294027017C2AF120BBA
:1010C0004478998664120ADF78988664D2AF120554
:1010D0004E412BC3E55294037017C2AF120B4478F4
:1010E000998664120AE578988664D2AF12054E415B
:1010F0002BC3E55294047017C2AF120B4478998643
:1011000064120AEB78988664D2AF12054E412BC365
:10111000E55294057017C2AF120B44789986641299
:101120000AEB78988664D2AF12054E412BC3E55284
:1011300094077019C3E5539406500201737401308B
:101140003A0274037888F6C238C239412BC3E5529B
:1011500094087019C3E55394065002017374023069
:101160003A0274047888F6D238D239412BC3E5525A
:1011700094097017C3E553940650020173303A0B7B
:10118000C37888E69402F6C23A412BC3E552940A2A
:101190007016C3E553940650020173203A0A78880A
:1011A000E62402F6D23A412BC3E55294147025C3CB
:1011B000E553940650020173C2AF901A0B7400936A
:1011C000D2AF7888F613C238C2394002D238400212
:1011D000D2398057C3E55294157038C3E55394064D
:1011E000404FC2AF901A0B740093D2AFF8B801020F
:1011F0007402B802027401B803027404B8040274E1
:10120000037888F613C238C2394002D2384002D27D
:10121000398018C3E552940C70117567A57568F193
:10122000C3E5539406400A911BD2AF755200755323
:10123000007567007568000173C2AF120B44E4D2F9
:10124000AFE4F55EF524F525F53D755E0812053E23
:101250001205A730EDFDA8BDA9BEE97001F8885FB1
:101260001205AB755E08C2AF120612855D5B855D27
:101270005CD2AF303A07C238303502D238D2287546
:101280003900120A84120AAF120621120628120629
:101290002112062812062112089F1209901209D85D
:1012A00012062812088F202C03120561302C03121D
:1012B0000591120990120A0312062812089F1209BA
:1012C00090120A2E12062812088F120990120A593B
:1012D00012062812089F120990120A841206281278
:1012E00005A712088F120990120AAF1205AB120659
:1012F00028302827855D5B79187A0CC3E539994039
:101300000EC228D2298A3B855D5B855D5C800CC35B
:10131000E5549401400302129761A130291F202B4C
:101320001CE53B147006C229D22A4197F53B203AAE
:1013300007C3E554940140030212978064753C0092
:10134000203A0F78FA79A4E760027803C3E555984C
:10135000504FE523604B303A172038052035078081
:101360000F303502800A202B07D22B855D5B41C7E9
:1013700078F0302B05855D5B7820C3E548985003F5
:10138000021297302B1BC22BC238303502D238D212
:1013900029753B12855D5B4197053CE55460026110
:1013A000A4753C00C2AF120B44752400752500D211
:1013B000AF12054E120B4478A4E6600CC290D29195
:1013C000C292D293C294D295C3E53C9404400302E6
:1013D0000DE1011E901A0D78209154E520B4550AB4
:1013E000A39154E520B4AA0280137567A57568F12E
:1013F000120B54911B756700756800801D901A03CD
:1014000078807B0A9154A308DBFA901A0F788C7BC2
:101410001A9154A308DBFA901A2922C2AF9197912E
:1014200074901A0074109159A374079159A37421F0
:101430009159901A0378807B0A9158A308DBFA909F
:101440001A0F788C7B1A9158A308DBFA91AA91881D
:10145000901A2922E493F622E6438F01538FFDFF71
:10146000C3E583941C400122EF8567B78568B7F018
:10147000538FFE22438F02438F018567B78568B77C
:10148000901A0DF0538FFC22901A0D7455915990BB
:101490001A0E74AA9159227A3079D07820901A4085
:1014A0009154E520F709A3DAF7227A3079D0901A1F
:1014B00040E7915909A3DAF9227C05120552DCFBB9
:1014C00022C2AF120AD9120ADF120AE5120AEB127F
:1014D0000546120AD9120ADF120AE5120AEB1205B2
:1014E00046120AD9120ADF120AE5120AEBD2AF221B
:1014F000C2AF120AEB120AE5120ADF120AD912056C
:1015000046120AEB120AE5120ADF120AD912054640
:0F151000120AEB120AE5120ADF120AD9D2AF2231
:1019FD00020D59100721FFFFFFFFFFFF09FF01FF38
:101A0D0055AA01FFFFFFFFFF03FFFFFF25D0285061
:0D1A1D0004FF02FF7AFF0701FFFF0000FF3A
:101A400023455F4C5F3030232020202020202020A1
:101A500023424C48454C492445464D3842313023B9
:101A60002020202020202020202020202020202076
:101C0000C2AFC2D37597DE7597AD7581C075A90057
:101C100043FF80752438752503B1DB7529A5752A26
:101C2000F143F12053A4DFD28575D4FF75E3407DE5
:101C3000FA780379E67C10752200752300901DE880
:101C40007B0675249875250130850281482085081A
:101C5000D8FBD9F9DCF781BA308508D8FBD9F9DC93
:101C6000F781BAB19BE493A3C39A6004DDC381BA40
:101C7000DBDBB18D600281317B08E493FAA3B16EA6
:101C8000DBF87A30B16E752200752300B18DEAFC65
:101C9000EBFDC3ED94FE400EB18D8A278B28ED300D
:101CA000E0048A828B83B18D7AC270D8C3ED94FE32
:101CB000601950CEBD0029EC600F7520007521FF22
:101CC000752900752A000200008100A827A92808AC
:101CD00009D804D90281DDB191EAF281D10D81A642
:101CE000C3ED94035051EDA2E092007AC5C3E582A2
:101CF0009400E583941C508C200010438F02438F86
:101D0000018529B7852AB7F0300027A827A9280818
:101D100009438F01538FFDD804D902A132C3E58353
:101D2000941C4003A3A117E28529B7852AB7F0A325
:101D3000A117538FFC81827AC1BD030CE493A3FAEF
:101D4000B152DCF8B14A81828184AA22AB23B16E00
:101D5000EBFAEA6222752608C3E52313F523E52290
:101D600013F52250066323A0632201D526EAB1DBD6
:101D7000B1DB75260AEAF4200102D285300102C2E5
:101D800085B1DBC3134002C201D526EB22B191EA33
:101D9000FB208502A191308502A196752608AE240C
:101DA000AF25C3EF13FFEE13FEB1DFB1DBC3EA13C0
:101DB0003085024480FA30E703632201C3E5231330
:101DC000F523E52213F52250066323A0632201D5F3
:101DD00026D9E52265236523F52222AE24AF250E00
:101DE0000FDEFEDFFCD20122424C48656C693437BD
:061DF0003164E8B10601B8
:00000001FF
